:020000040000FA
:020000002E28A8
:08000800F1000308F2000408F6
:10001000F30083010B1D1028210885000B112728F0
:100020008C1E272806301805031D182818121816CC
:1000300043080F3A031D1E28C301B20132304307A3
:1000400084001A088000C30A840A800127287308E4
:10005000840072088300F10E710E0900830185018E
:10006000860107309F0083168501FB3086008117CB
:100070008C1683128B170B178316193099002630B4
:100080009800831290309800A201B201C201C3010E
:10009000D301CF0122304207840003308A00420896
:1000A00000238000800803195828840AC20A4D28BA
:1000B0000514FD20A201C20105100921061C5E28BD
:1000C00006186028D4012621D40A0319D403061C7B
:1000D00063285408103C03185E2885144B308400B4
:1000E0000430D50080010830CA00800D061876283B
:1000F0001D21061C800A2621CA0B7528840AD50BEF
:1001000072288510D5014B30550784000008D600B1
:100110004F30550784000008D602031D9928D50AE0
:1001200004305502031D83280514D30A0319D30391
:10013000AB280510D301D5014B30550784000008CA
:10014000D6004F305507840056088000D50A043089
:100150005502031D9C285308033C031D5E284B08D1
:10016000AA3C031D5E284C08D1202030C7204D0832
:10017000D1204E08D120BC280A30C7200D30C7201E
:100180000030C720FD20A201C2015E282E28C40035
:1001900022304207840044088000C20A840A800199
:1001A0000800C4002230420784000230C500C40E9B
:1001B00044080F39C600303E8000393C0318E2285D
:1001C00007308007C20A840AC50BD72880010800BF
:1001D000C4002230420784000830C500C40D031C4F
:1001E000F3283130F42830308000C20A840AC50B6D
:1001F000EE28800108003230FE28223084000008FA
:100200000319080099008316981C04298312840A94
:10021000FF280530C900C801C701C70B0D29C80B4D
:100220000C29C90B0B2908000530C8004130C70054
:10023000C70B1829C80B162908000130C8009D30CB
:10024000C700C70B2129C80B1F2908002D30C80083
:0E0250000130C700C70B2A29C80B2829080057
:10060000820743346F34753463346F3475340A347D
:040610000D34003471
:02400E00013F70
:00000001FF
